:10000000830100308A0004288301C8298312BC00C0
:10001000BD1B11283D088A003C08BC0A0319BD0A13
:10002000820083133D1883173C08BC0A8400000833
:1000300008000C3448344F344F3444344D34493480
:10004000433452344F342034533465347234693479
:1000500061346C3420344234693474346234613431
:100060006E34673420344534783461346D34703400
:100070006C34653400340A340D342534643400346F
:100080000A340D3443346F34703479347234693443
:100090006734683474342034283463342934203489
:1000A00032343034303435342C3420344B34393419
:1000B000733470347534643420344C344C344334E9
:0200C00000340A
:1002FA0000300B2AB5000030361835070310B50D4B
:10030A000310B60CB608031908008129B901BA010D
:10031A000310B80CB70C031C99293508B90736081D
:10032A000318360ABA070310B50DB60D3708380494
:10033A00031900348D29B300F730B4008B13050874
:10034A0004388500BE21BC21B40A0319B529B30CAF
:10035A00031CA529FB3900008500BC21BF21A9295E
:10036A00B629FB3985008B17BE21BE210800000083
:10037A00C029BF29C029C129C229C329C429C5291D
:10038A00C629C72908008312A0018B01EB30831606
:10039A0085008312FF2383169000831205161930F5
:1003AA00A6000030A7007D214030A6000030A7003B
:1003BA007D210512A101A201E229A10A0319A20ABB
:1003CA0027302202103003192102031CED29EE29DD
:1003DA00E2290516A101A201F229A10A0319A20A1A
:1003EA0027302202103003192102031CFD29FE299D
:0603FA00F2293B30A600D1
:100400000030A700A00A2008A300A4012330A50003
:100410007D21DE2904288312AE00AC012508A90045
:10042000B22B2D08253A031DA52BFF30AA00AB01E6
:10043000A8016F2BAE080319202A2E088400800122
:100440002C0808000230A907290284000008A32B09
:10045000A80A2E2A0830AA07FE30AA070230A907E8
:10046000290284000008AF00840A0008B0002818A0
:10047000B01F412AAF09B009AF0A0319B00AAB0394
:10048000422AA8010B30AA072A08B700B801300891
:10049000B6002F08B500C5233508AD002A08B700FF
:1004A000B8012F08B5003008B600C5233908AF00E1
:1004B0003A08B000B101B10AB20132083002031D9E
:1004C000632A31082F02031C802A2A08B700B801CA
:1004D0003108B5003208B6008B213908B1003A085E
:1004E000B200AB035D2AAC0AAE0803197D2A2E08C0
:1004F000840020308000AE0A802A20308312A021A0
:10050000AB032B08803A7F3E0318732A281C932ADA
:10051000AC0AAE080319902A2E0884002D30C32A95
:100520002D308312A0212A08B700B8013108B50088
:100530003208B600C5233908B1003A08B2003104C8
:100540000319C92A3208B8003108B7003008B600CC
:100550002F08B500C5233908B5003A08B6002A08A7
:10056000B700B801C5233508AB00803A763E031CBE
:10057000BB2A0730AB07AC0AAE080319C62A2E08FF
:1005800084002B08303E8000AE0A932A2B08303EB0
:10059000912A0A302D02031CCF2A0730AD07AC0A7E
:1005A000AE080319D82A2E0884002D08303EAC2B43
:1005B0002D08303EB02BAC0AAE080319E52A2E08F0
:1005C000840020308000AE0AE82A20308312A02167
:1005D000AB032B08803A7E3E0318DB2A0230A907C2
:1005E000290284000008AD00A52B0230A9072902CA
:1005F00084000008B100840A0008B200AD012D0893
:100600003107BC003208BD003C080318BD0A0620B3
:10061000003803190D2BAD0AFF2A2A082D020318F2
:10062000132B2D08AA002A08AB1B3E2BFF3A2B07E1
:10063000031C3E2BAC0AAE080319242B2E088400A1
:1006400020308000AE0A272B20308312A021AB037C
:10065000132B3208BD0031080620AD00B10A031982
:10066000B20AAC0AAE0803193B2B2E0884002D08F1
:100670008000AE0A3E2B2D088312A021AA032A0F68
:10068000292BB22B2708BD00260806202A3A031D75
:100690004F2B0230A9072902840000086B2B270882
:1006A000BD0026080620D03EAA00A60A0319A70A04
:1006B0002708BD0026080620AD0030302D02031C9F
:1006C0006F2B3A302D0203186F2B0A30B6002A0820
:1006D0007F212D07D03EAA00A60A0319A70A2708E2
:1006E000BD002608A60A0319A70A0620AD00003A95
:1006F00003191A2A2A3A0319222A043A0319422B07
:10070000763A03192A2A3B3A0319E92A073A0319C8
:10071000282A0B3A03192C2A1C3A0319F52A063AFF
:1007200003192E2A0D3A03192A2A30302D02031CF0
:10073000A52B3A302D020318A52B0A30B6002B0842
:100740007F212D07D03EAB006F2BAC0AAE080319FA
:10075000AF2B2E0884002D088000AE0AB22B2D0886
:100760008312A0212708BD002608A60A0319A70A9C
:100770000620AD00AD08031D112AAE080319C32BD6
:100780002E08840080012C080800BB01B901BA01C1
:1007900037083804031DCF2BB501B60100341F30D4
:1007A000BB040310BB0AB70DB80D031CD22BB80C49
:1007B000B70C38083602031DDF2B37083502031C3F
:1007C000E72B3708B5023808031C380AB602B90D02
:1007D000BA0DBB0BBB1AD72BBB1FF32BB909B90A38
:1007E0000319BA03BA093908B7003A08B8003B1F21
:0E07F0000034B509B50A0319B603B609003482
:02400E00E43F8D
:00000001FF
